:020000040800F2
:1050000034483349016034494160344901613449CD
:1050100081603449C1603449416134498161344916
:10502000016234494162344981623449C162344980
:105030000163344941633449C1633449816334496C
:10504000C16134494164344981643449016434495B
:10505000C164344901653449416534498165344945
:10506000C165344901663449816634494166344931
:10507000C16634490167344941673449C1673449DD
:105080008167803033490160334941603349816031
:105090003349C16033490161334901623349416297
:1050A00033494161334981613349C1613349016306
:1050B000334981623349C162334941633349816372
:1050C000704710B500F064FB00F02EFC002010BD0E
:1050D000176200087405002031760008D595000895
:1050E000A9760008C3830008796700087771000873
:1050F000CD5100084B65000849670008E199000898
:10510000D75E0008D379000865520008E351000813
:105110005F550008C15B00088B7B0008BB75000869
:105120006D7500085554000805550008936D00087A
:1051300011760008A9560008455F00087D5D00084B
:105140009356000853980008975E0008035600081D
:105150004F6300086B7600084771000875840008EB
:10516000C78400081D850008C5950008755E000805
:105170003F740008259500085D5D000879860008E9
:10518000BF7400086795000849850008819A0008E7
:10519000302802D94FF0FF307047A74A202802EB91
:1051A000800202D922F8821C0EE0102806D952F89B
:1051B000440D00F0FF1040EA012004E052F8040D15
:1051C0009E4B184008431060002070479A4A002008
:1051D0006FF07F4142F82010401CC0B20F28F9D96F
:1051E0007047F0B5401EC4B2601E0D46302802D391
:1051F0004FF0FF30F0BD924F0A26A7F1240C95FB2B
:10520000F6F006FB105095FBF6F5C1B2385D641E52
:10521000E4B21CF80110FFF7BBFF002DEFDC00200B
:10522000F0BD8749A0F141023E390144192A02D854
:1052300011F9410C7047A0F16102192A02D811F945
:10524000610C7047A0F13001092901D848B27047BC
:105250002D2803D02E2803D023207047212070470B
:1052600022207047F0B5764F00250E460446243FB5
:10527000DFF8CCC112E0FFF7D4FFC0B2395C0CEB11
:10528000040010F8010CFFF783FF641CE4B2302C1B
:1052900002D94FF0FF30F0BD6D1CEDB2705D0028FB
:1052A000E9D1F0BD70B5044663480D464030FEF7C5
:1052B0005DFE2846FEF77EFE6149C0B246390123F5
:1052C00088704D7900222DB12044401EC8704A706C
:1052D0000B7103E0CC70401E48700A714A718A71EC
:1052E000CB710B7070BD2DE9F0470346FFF76EFFE1
:1052F000DFF84CA1DFF84C91AAF1240AF3B34FF088
:10530000000800252FE0002425E04D4FD4461AF870
:105310000510385DFFF73CFF3E191CF8051016F824
:10532000100FFFF735FF1CF80510307CFFF730FF3A
:10533000C82004F0F7F8385DFF21FFF729FF307827
:10534000FF21FFF725FF307CFF21FFF721FF641CC1
:10535000E4B20F2C03D899F800000028D5D06D1CBA
:10536000EDB21E2D03D899F800100029CBD008F11A
:10537000010000F0FF08B8F10F0F00E001E0C0D914
:105380002EE0002556464FF4C8784F46002420E012
:105390004FF0010C315D6046FFF7FAFE0CF1010C95
:1053A0000CF0FF0CBCF1300FF4D9404604F0BAF811
:1053B0004FF0010CFF216046FFF7EAFE0CF1010CF3
:1053C0000CF0FF0CBCF1300FF4D9641CE4B21D2CBE
:1053D00002D838780028DBD06D1CEDB2282DD5D945
:1053E00099F8000010B9184901200860FFF7EEFE97
:1053F00016490120FFF736FFBDE8F04714490720A2
:1054000030E7704710B50C4C0021403400F00F021B
:10541000C1F105030009E254092A01D9413200E033
:105420003032491CC9B2E2540629EFD30020A071E2
:105430000148403010BD0000BC0A002000FFFF0002
:10544000530200202C09002030090020BC08002055
:10545000D808002070B5AD4D420730D50C0901F0D9
:105460000F01820702D5285D484005E0C00705D03E
:10547000285DC1F10F010840285500E02955A44ED0
:105480003088C00705D03188C807FCD1052004F05A
:105490006AF8A048C1684FF60F7211402A5D41EAD0
:1054A0000211C1609C480168C1F30A0141EA04315C
:1054B000016001213046FBF7AFFA002070BD3129B1
:1054C00002D94FF0FF3070BD4A1ED31702EB937222
:1054D000C2F3870422F00302491E8A1A0121914077
:1054E000C9B2C20702D0285D084307E08007285DE3
:1054F00001D5484002E0C1F10F010840285500F0F5
:105500000F00B9E72DE9F0478448804EDFF80082AC
:10551000DFF80092804F056800244FF60F7A315D66
:1055200015F8010B0143315540460288D207FCD1E2
:10553000D9F80C2002EA0A0242EA0111C9F80C105B
:105540003968C1F30A0141EA043139600121FBF7EE
:1055500063FA641CE4B20C2CE1D3BDE8F0872DE9BA
:10556000F0476E48694EDFF8A881DFF8A8916A4FCE
:10557000056800244FF60F7A15F8010B315DC0F174
:105580000F000140315540460288D207FCD1D9F8BE
:105590000C3003EA0A0343EA0111C9F80C10396818
:1055A000C1F30A0141EA043139600121FBF734FA01
:1055B000641CE4B20C2CDFD3CFE7411ECA1701EB09
:1055C000927230B5554901240B6803EBA20209E041
:1055D000312814D0401CC0B2411ECA1701EB927191
:1055E00003EBA102411ECD1701EB957525F00305D4
:1055F0001278491B04FA01F10A42E9D030BD0420B7
:10560000EAE72DE9F0410024444E14270B20FEF771
:105610008AF8401C05B21020FEF785F83168495D14
:10562000014041EA0510C1B20420FFF713FF142026
:1056300003F099FFB4FBF7F007FB104008B9FFF740
:1056400061FF641CC82CE1D3BDE8F0812DE9F0476F
:105650000024DFF8B8902E4F2E4D2F4EA0464FF667
:105660000F7A09F8048038460188C907FCD1E96837
:1056700001EA0A01E9603168C1F30A0141EA043133
:1056800031600121FBF7C8F9641CE4B20C2CE8D3AB
:1056900063E71E49002001F10C020B5C1354401C0F
:1056A000C0B20C28F9D3704770B5184D00240C35E2
:1056B000285D40EA0410C1B20420FFF7CBFE641C51
:1056C000E4B20C2CF4D370BD70B5154C4FF4967049
:1056D0004FF4FA76134D20600FE0FFF713FF3046CA
:1056E00003F020FFFFF73BFF287810B9304603F0A6
:1056F00019FF2168491E216002D028780028ECD0CB
:105700002878002801D10120206070BD150B0020F1
:1057100000040040001001400C0C01409C080020D7
:10572000300900202C09002070B5D34D0420D34946
:10573000E87002200870D24800240470D148047038
:1057400003F07FF9D149D0480860D1490860D148B9
:105750002C70AC70047070BD10B5CE480024CEA182
:1057600004700120FFF77EFD03F04AFBFDF7FDFC0E
:1057700020B1CBA10120FFF775FD01E0FFF726FD69
:10578000C948BE49046002200870C848047010BDB2
:1057900070B5C748016841F4E0210160C5484FF485
:1057A0007A76C5490660C8200870C4490F200025D4
:1057B0000870B24902200870C1480570FDF737FD36
:1057C000FDF7B2FDFDF77FFDFAF7C0FEFDF714FD12
:1057D000FDF7BEFEFDF707FEFDF72DFEFDF75AFEB5
:1057E000FDF783FEB7480124C0F8AC41FFF708FC81
:1057F000FFF72CFF00F00BFAFFF7E8FCB249C1F805
:105800009441C1F8984100F066FBFDF7FAFCFBF704
:1058100086FE30B9FBF7DDFC0120FBF71AFEFBF733
:10582000DEFCFDF78AFF03F060FF03F0BAFEFFF72E
:105830007BFFFDF7B4FD0020FDF780FC9548007864
:10584000401E0B2802D30020FFF786FFFDF701FC66
:1058500030B19EA10120FFF705FD304603F083FE25
:105860000020FDF776FC904C9C4E2168884201D1C7
:10587000307878B39AA10120FFF7F4FC9AA10720B1
:10588000FFF7F0FC03F025F835700020FDF761FC10
:105890002060FDF76AFC4FF4487003F064FE0020BE
:1058A000FDF757FC2168884212D091A10120FFF733
:1058B000D9FC91A10720FFF7D5FC4FF4C87003F085
:1058C00052FEFDF73AFF642003F04DFEFDF735FF71
:1058D000FFF77CFC8A48008881B28A48007804F08F
:1058E000CFF88948008881B28848007804F0C8F869
:1058F00087480068804701F0F6FB86A10120FFF78A
:10590000B1FC86490920FFF7ADFC85A11120FFF706
:10591000A9FC594881681920FFF7A4FCBDE8704034
:105920004FF4FA6003F01FBEDFF8FCB17F4F574E13
:10593000DFF84891DFF8F8A14FF000084E4CE0780E
:10594000012801D0022819D12079032814D37948DD
:105950006C4900680978007A88420DD07649FDF7D5
:10596000B5FE76A17A48FEF701FB73497848FEF749
:1059700040FB7748FEF77FFA03F0AFFF444D3168F4
:105980002868884256D000F0C1FA6070FF2851D0D4
:10599000217979B100F0AFFA6749FDF797FE6DA163
:1059A0006B48FEF7E3FA64496948FEF722FB684852
:1059B000FEF761FA6078A0F17001072901D8012192
:1059C00000E000218BF8001099F80020022A03D093
:1059D00029B102F058FF1DE00029FAD11AE000F0C9
:1059E00081FA61490968884700280BDA6178FF2944
:1059F00008D05E48426842F47F4242601620FFF7BA
:105A0000F0FB05E02079012802D159A0FEF733FA16
:105A10008AF80080387850B95F48007803F0A3FD19
:105A200028683168884202D0607800F08BFA87F8E5
:105A30000080A4E799F8000001280BD19AF8001023
:105A400050462D2906D380F80080207910B153A04C
:105A5000FEF711FA574C207848B1574D28780128A5
:105A600005D1FEF77FF985F8008084F8008053485F
:105A70000068804762E70000CC030020DD060020BC
:105A8000510300202C090020930B002074060020F5
:105A90007006002048040020202067616D6500002A
:105AA000206572726F720000B00400209E06002014
:105AB00024ED00E0780400202D04002042040020A2
:105AC0008B0800200080214200002342736574751A
:105AD0007020206572726F72200000003804002070
:105AE00020726573657400006E7672616D2000002F
:105AF000206E7672616D000073686F742020000064
:105B00007C0400207407002080040020EC070020A3
:105B10008C02002020702D7265760000DE060020C9
:105B200020672D72657600009A060020A2060020EC
:105B300005090020340900202D0B00204576656EF4
:105B4000742074726967676572202D200000000060
:105B5000230C002053776974636820436C6F73656E
:105B600064202D200000000084020020BC0A0020D8
:105B7000537769746368206E6F742070726F6772F8
:105B8000616D6D656420666F72207468697320674B
:105B9000616D653F213F0000340800205761746348
:105BA00068646F672042616C6C2053656172636842
:105BB0002E0000000409002000000020C002002088
:105BC00030B40346092904D9002B1ED0B1F5007F5B
:105BD0001BD25A480288D207FCD1594ADC0709D0A7
:105BE000146884EAC1141460022B0AD230BC01216B
:105BF000FAF712BF0124891D04FA01F114684C4020
:105C0000F1E7504A10884840108030BC70474C483B
:105C100001684FF6807211430160704710B5044669
:105C200003F056F808B1012010BD21462E20FFF7E1
:105C3000D8FA21460220FFF70DFC4FF4967003F0CE
:105C400092FC21460220FFF705FC4FF4FA7003F0A6
:105C50008AFC002010BD2DE9F041012100260846F4
:105C6000FFF7F8FB012455E037A12F20FFF7FAFAE0
:105C70000025364FDFF8D8800AE03868405DFFF72E
:105C8000CDFF03F025F838B900F025F96D1CEDB211
:105C900098F800008542F0D32EA12F20FFF7E2FAFA
:105CA0002CA12D20FFF7DEFA03F012F8B0BB01257E
:105CB0004FF4FA674FF4487823E029462E20FFF787
:105CC00090FA29460020FFF77BFF0EB1384600E02E
:105CD000404603F048FC00F02BF9742801D126B1AE
:105CE000002602F0F5FF88B901E00126F9E700F08F
:105CF000F2F816B1641CE4B201E06D1CEDB2092D9E
:105D000004D802F0E5FF08B9142CD6D3641CE4B221
:105D1000142C03D802F0DCFF0028A5D002F0D8FF35
:105D200010B90D490120086001210020FFF792FB06
:105D3000BDE8F04107A12D20FFF794BA000800400C
:105D40000C180140300600204C530000A008002031
:105D50008B080020202000003009002010B50F29FA
:105D60000BD83B4CE0680843E060282003F0FBFBC5
:105D7000E0684FF6F0710840E06010BD70B5054670
:105D80000C46052902D13348007818B9324800780A
:105D9000002818D03148007800B102250F2C0ED908
:105DA0000A210120FFF756FB04F00F012846FFF7F8
:105DB000D5FFBDE870400A210020FFF74BBB284605
:105DC000BDE87040CAE770BD2DE9F0470124DFF857
:105DD0009090244FDFF89080254600264FF47A6A91
:105DE00022A12D20FFF73EFA21462E20FFF7F9F9D8
:105DF000012D03D121460020FFF7C0FF504603F0DC
:105E000091FB99F80000A8B1454638682968884296
:105E10000ED000F07BF8742803D07028F5D101264D
:105E2000F3E71F2C02D0641CE4B2EEE70124ECE798
:105E3000012501E06D1CEDB226B9142DD0D30C491B
:105E400001200860BDE8F04708A12D20FFF70ABA3D
:105E500000100140390400203A04002032060020DE
:105E60002C0900207006002074060020202000006D
:105E7000300900200A21B0FBF1F201FB1202B0FB55
:105E8000F1F1C44B012088409A5C024201D000200D
:105E900070470120704730B5BE4CBF4B0C3C2246CA
:105EA000A16852684FF0FF35994201D13F3B00E0B5
:105EB0004B1C9A4201D1284630BD08700020A360D7
:105EC00030BDB4480C38D0E90110814201D0012026
:105ED000704700207047B048AE493F380C398860A1
:105EE0004860704700F00F01000900EB800001EBF3
:105EF0004000C0B270470A21B0FBF1F201FB120270
:105F0000B0FBF1F002EB0010C0B27047A14A0C3AAE
:105F1000D2E90110814201D1FF2070479E4B0878E1
:105F2000994202D1A3F13F0100E0491C5160704742
:105F300098490C39D1E90101884201D1FF2070470D
:105F40000078704730B5934C934A0C3CFF2361684E
:105F500009E00D78854200D10B70914202D18E4943
:105F60003F3900E0491CA568A942F2D130BD70B5A7
:105F70008A4C0546207840B1894E3078012804D1FA
:105F8000FDF7F0FE002030702070824C0C3CD4E90C
:105F90000101884208D1284603F0C4FAD4E901017E
:105FA000884201D1FF2070BDBDE87040AEE770B5FA
:105FB00000254FF416763046FFF7D9FF04467028C7
:105FC00007D0742C05D06D1CEDB23C2DF3D300200E
:105FD00070BDC820FFF7CBFF702807D0742802D00F
:105FE000702C0BD006E0702C06D003E0702C05D08E
:105FF000742C01D0012070BD022070BD032070BD43
:1060000070B500254FF496763046FFF7B0FF044692
:10601000FF2804D0702C07D0742C05D01CE04A2037
:10602000FFF728FFC0B174244FF4C870FFF79FFF3B
:10603000702807D0742802D0702C0BD006E0702C8A
:1060400006D003E0702C05D0742C01D0012070BD67
:10605000022070BD032070BD6D1CC82DD4DB002054
:1060600070BD10B5FFF7A3FF4E49087010BD10B505
:10607000FFF7C6FF4B49087010BD464A0A210C3A8B
:106080001078B0FBF1F301FB1301052901D0401C8E
:1060900002E04B2802D0401D107070470020FBE743
:1060A0002DE9F047DFF8EC900025A9F10C09DFF8A5
:1060B000F8A03E4EDFF8F8805AE04FF44870FFF742
:1060C00056FF044670280DD0742C06D025B34C46DC
:1060D0002078FFF7CFFE58B10DE00DB1002547E065
:1060E000012545E00020386042E0FFF7C6FFEFE7FA
:1060F00020780028F9D132682EA115209047217808
:1061000029B11620FFF76DF8FFF7B7FF30E0012047
:10611000207028A1162029E0FF2C37DAFFF7E2FED5
:1061200001461620FFF75DF81420FFF720FFA0427C
:106130001ED1214F0124326820A1012090473268EE
:10614000514607209047FA2003F00DFA386880473F
:10615000642003F008FA641C042CECDDFFF7BBFE9E
:10616000326818490120904751460720326890470D
:10617000D8F800004746401EC8F80000401C9CD1DB
:106180003268BDE8F04710A1152010470FA1152077
:10619000ECE7000078060020D20B00200409002064
:1061A00000000020BD060020ED080020B005002002
:1061B000300900202000000094050020636C656118
:1061C0006E200000BC080020202000002D2D0000C3
:1061D00070B5FB4CFB4D20782978884201D300290B
:1061E00018D1632816D2401C207005210220FFF729
:1061F000C5FD287820B920780F2801D90F202070FC
:10620000F1480078002805D02178BDE870403020A2
:10621000FEF7E7BF70BD70B5EC48ED4C007894F820
:106220002610884218D9EB480125007868B9042166
:106230000120FFF70FF9E57594F82600401C84F85B
:106240002600E5480168491C01602576BDE87040DC
:1062500002210846FFF792BD70BDD94A1078002888
:1062600009D0401EC1B2D84811700078002802D071
:106270003020FEF7B6BF704770B5D54C0025607E64
:1062800020B1657602210020FFF7E4F8D3480078BA
:1062900003F0A6FBD2480068804720B14FF4FA60B3
:1062A00003F061F901E0FEF791FFCC483038007847
:1062B00003F096FBE57084F82650022084F8450030
:1062C00001202070E574BDE8704000F040B8C5487A
:1062D000007800280BD0BE4A002100EB400011716D
:1062E00002F18001C86101F1680003F0B2BA7047A1
:1062F000B749002001F1800281F8280081F82900C7
:10630000106350639063D06301231064CB7688667A
:1063100081F83900C866086781F83A0048678867DD
:1063200081F83B00C867106081F83C00506081F83C
:106330003E30C87081F82B0081F8360081F82600C5
:10634000A94B13618875C87581F84000704770B516
:106350009C48007818B19A48007800287DD09C4C61
:106360000025012694F8451002291BD094F83E0020
:10637000012872D1E07E01286FD12046082990F8CB
:10638000360073D0012968D1E17C002967D0217DD6
:10639000002965D0042860D204F5A470007803F0C9
:1063A0001FFB65E08E48A67400688047217808438B
:1063B00053D08A4825702438007803F011FB8748B1
:1063C0001830007803F00CFB84486038007803F044
:1063D00007FB82485438007803F002FB7F484838B6
:1063E000007803F0FDFAA574FEF7F0FE7F48006820
:1063F00080477F4800688047082084F845000121D5
:106400002E20FEF7EEFEA5710B210020FFF722F8EB
:1064100004210020FFF71EF801210846FFF71AF8B3
:106420000C210020FFF716F802210020FFF712F8D8
:10643000FFF75EFF6F4800688047FFF790F86E48EF
:1064400000688047FFF747FD6C4861490068E066D7
:1064500060678031E067486003E02EE006E027E0F7
:1064600023E0FFF734FFE574257506E0042824D205
:10647000E57404210020FFF781FCFFF7EEFE14F81D
:10648000360F5F49401CC0B220700A68521C0A6077
:10649000012813D0022814D003284FF0000113D094
:1064A0001C20BDE87040FEF79CBEBDE87040E3E6EE
:1064B0004A480C3803F0CDF9E67470BD002106207F
:1064C000EFE700210C20ECE71620EAE7444810B57E
:1064D0000068804700280ED03D48817C00290AD002
:1064E00090F84500022806D146A10720FEF7BAFE23
:1064F000BDE810402BE710BD70B5354C04F18000AD
:10650000E17811B1C169491EC161C069012528B195
:10651000607978B10020607104210EE094F82600C3
:106520004FF0040120B10120FEF794FF257170BDEA
:106530000020F9E7657104210120FEF78BFFBDE81B
:10654000704026486C3803F084B9214A1046117F08
:10655000407F1429084407D301D1D07F01E0A0F186
:10656000150082F82A0070470A2905D301D1907FCF
:10657000F7E7A0F10B00F4E7A0F10100F1E710B597
:1065800008210020FFF71CFB20480D4A0168491C28
:1065900001600C4910780978884201D300290DD197
:1065A00063280BD2401CC1B2074811700078002844
:1065B00004D0BDE810403020FEF713BE10BD00002F
:1065C000450400204304002034040020440400203B
:1065D000980600202204002068040020EC07002018
:1065E000A40200202604002040420F009002002058
:1065F000A0020020B0020020AC0200208404002091
:1066000058040020202020202020000070040020BA
:10661000FE4810B500780028D0D0FFF7B0FFBDE8E5
:1066200010404FF4967002F09EBFC7E72DE9F0418D
:10663000F748F84D007840B9F749E86C884204DD26
:1066400090FBF1F201FB1200E864F44CE86C216865
:10665000884224DDF24E307808B1FFF7D9FFF14FC0
:10666000E86C396888421CDD2160EF4C2168884263
:1066700014DD307808B1FFF7CBFF20683860EB4FAE
:10668000E86C396888420CDD2160FFF7C1FF307883
:1066900018B9FFF7BDFFFFF7BBFFE86C3860BDE836
:1066A000F0812060FBE70246491EC8B2D9490123A8
:1066B00080310F2A05D0082A16D90E2A08D020B119
:1066C00013E090B903204B61704702F0070006E029
:1066D00040B9D04890F84500012803D00220486115
:1066E000022070474B6105E010B100224A617047FB
:1066F000521C4A6101207047CD480068004710B520
:10670000C44CE07800281ED10120E07094F82600E7
:1067100028B904210020FEF79DFE0020E075C54841
:10672000007800280FD0E07A08B1607A01E0617A41
:1067300019B110B9BE4800688047BF480078BDE86D
:10674000104003F04DB939E7B24810B5014690F852
:106750002540897801220023012C02D019B142651D
:1067600002E039B183704365416DC164C0E918230B
:10677000C26523E78270F2E7A64890F82510012948
:1067800001D0C16C01E0816DC1644165012110221D
:10679000C0E91821C1657047082805D90E2801D223
:1067A000022070470F2801D0012070470320704756
:1067B0002DE9F047974D0024012785F8254010204A
:1067C00085F83770DFF87482DFF8749285F8380046
:1067D0000F26AFF2D0110720FEF744FD95F83700E1
:1067E000012814D197A1FEF73DFD98A10720FEF7DF
:1067F00039FD984B1878E864FFF7BEFF95F84C0018
:106800001870FFF7C9FF85F83200C5E9186495F8DC
:106810003700022815D190A10120FEF723FD8BA19E
:106820000720FEF71FFD8E4B1878E864FFF7A4FFE2
:1068300095F84C001870FFF7AFFF85F83300C5E9F5
:10684000186495F83700032815D186A10120FEF7BA
:1068500009FD7EA10720FEF705FD844B1878E8644A
:10686000FFF78AFF95F84C001870FFF795FF85F841
:106870003400C5E9186495F83700042811D17CA1CB
:106880000120FEF7EFFC7CA10720FEF7EBFCDFF810
:10689000F0C19CF80000A870FFF756FFA8788CF8AC
:1068A000000095F83700052811D176A10120FEF7E8
:1068B000D9FC76A10720FEF7D5FC764B1878E86462
:1068C000FFF75AFF95F84C001870C5E9186495F861
:1068D0003700062811D170A10120FEF7C3FC70A17A
:1068E0000720FEF7BFFCDFF8C0C19CF80000A870CD
:1068F000FFF72AFFA8788CF8000095F837000728E2
:1069000011D16AA10120FEF7ADFC6AA10720FEF7B4
:10691000A9FCDFF8A8C19CF80000A870FFF714FFDD
:10692000A8788CF8000095F83700082811D164A1E8
:106930000120FEF797FC53A10720FEF793FCDFF838
:1069400088C19CF80000A870FFF7FEFEA8788CF8BC
:10695000000095F83700092811D15CA10120FEF74D
:1069600081FC5CA10720FEF77DFCDFF870C19CF87C
:106970000000A870FFF7E8FEA8788CF8000095F8F2
:1069800037000A2819D151A10120FEF76BFC54A150
:106990000720FEF767FC95F82500012802D1A96DB4
:1069A000C8F80010D8F80000E86468654FF47A7001
:1069B0004EF66021C5E91810E86595F837000B28F8
:1069C00011D149A10120FEF74DFC35A10720FEF7AA
:1069D00049FCDFF81CC19CF80000A870FFF7B4FE6A
:1069E000A8788CF8000095F837000C280CD141A14C
:1069F0000120FEF737FC20A10720FEF733FCDFF86B
:106A0000FCC09CF800007BE080E000003604002021
:106A1000350400209806002040420F008804002022
:106A200032040020A80400209C0400208C040020D4
:106A3000D40200203B040020F8070020A00400201E
:106A4000A608002020206C6566740000636F696EE4
:106A50007300000029040020207269676874000038
:106A60002A04002063656E74657200002B04002008
:106A700020636875746500006D61746368000000D0
:106A80002804002063726564697400006C696D6994
:106A900074000000430400202020636F696E000032
:106AA000736F756E647300003904002020207368D2
:106AB0006F77000063726564730000003404002087
:106AC00073706563696100002F0400207370656353
:106AD000696C00006F766572726400002E040020FD
:106AE00061776172640000002073636F726500005B
:106AF0003A040020656E61626C650000310400207C
:106B0000A870FFF721FEA8788CF8000095F83700F0
:106B10000D2812D1FEA10120FEF7A4FBAFF29401D3
:106B20000720FEF79FFBFC4B1878E864FFF724FE74
:106B300095F84C0018700820286695F837000E2844
:106B400011D1F6A10120FEF78DFBF6A10720FEF77B
:106B500089FBDFF8D8C39CF80000A870FFF7F4FDAC
:106B6000A8788CF8000095F837000F2812D1AFF202
:106B70007C010120FEF776FBEDA10720FEF772FBFA
:106B8000DFF8B4C39CF80000A870FFF7DDFDA8781B
:106B90008CF8000095F8370095F8381088420FD12E
:106BA000E6A10120FEF75EFBE6A10720FEF75AFBF7
:106BB0004FF0FF30EC65E86495F82500012819D006
:106BC000AFF2C0511120FEF74DFBE96C002902DB4A
:106BD0001620FEF706FBDD49886C401E886409D04C
:106BE000FFF7E5F985F8250001280ED0022819D015
:106BF00003281CD0D6A10120FEF734FBAFF2FC51D4
:106C0000BDE8F0470720FEF72DBBD5E917010A1AAA
:106C1000696D8A4201DA686E00E00844A86589F867
:106C20000070D6E5686EA86585F82570F7E795F8D9
:106C3000370095F83810884202D185F83770C8E5DA
:106C4000401C85F83700C4E5C34810B5006880478C
:106C50000C21BDE810400120FEF7FCBBBB48002121
:106C6000803800F8281F4170B8485C3002F0F1BD50
:106C700030B5B649B948A1F18004CA68006894F8F3
:106C80003610B74B50B1884208D91D68411A694384
:106C9000B1FBF0F1B2FBF0F2114401E092FBF1F133
:106CA0001960B0490A78002A2DD0AF490A2809682E
:106CB00002D8B1EB500F26D964256943B1FBF0F13E
:106CC0002165881A1B686430584390FBF5F042F246
:106CD000107390FBF3F05843A44B984200DDA44896
:106CE000914210D0A34900EB0012A34B08600A2187
:106CF00092FBF1F21A6000EBC00202EB001090FB75
:106D0000F1F09E49086030BD70B5904D0120A5F1AD
:106D100080046861A06E6426E06490FBF6F106FBD7
:106D20001100A86194F82B10884201D1FFF727FCCD
:106D30006869401C686194F8361088420AD80228B5
:106D400004D0032804D02868E064E6E7206FFBE75E
:106D5000A06FF9E770BD10B57C4C0020803CA07698
:106D6000AFF260710120FEF77DFAAFF26871072083
:106D7000FEF778FA0620A16EFEF733FA94F8360093
:106D8000012805D9216FBDE810400C20FEF729BA73
:106D900014E42DE9F0476D4C803C94F8450002283E
:106DA0007DD02046E1780079002504F5AA790126F6
:106DB00001B110B9617E002972D0A07E58B163483C
:106DC0009830007802F00CFE6048A430007802F0A1
:106DD00007FEFFF7C0FF6A4800688047607EA0B1E9
:106DE000657602210020FEF735FB84F84560AFF29E
:106DF000EC716448FDF7BAF862492C20FEF732FACC
:106E000060492620FEF72EFA02E05F4800688047BE
:106E100099F8000002F0E4FDE57094F826004B4F6D
:106E200018B1401E84F826001AE094F83E0094F849
:106E30003610884211D15549E07E0978884208D23F
:106E4000401CC1B2E1762E20FEF7CBF984F83E60FB
:106E500006E0022084F8450023E0401C84F83E0050
:106E600094F8450002281CD0207A00284ED0DFF884
:106E700020810620D8F80010FEF7B3F945480078C5
:106E8000002844D0444801680C20FEF7AAF9434882
:106E900001681620FEF7A5F941480168A9E020E144
:106EA000E6E001210020FEF7D5FA3E480078A8B1BF
:106EB0000A207861FCF737FC397D4843C1B284F879
:106EC0002B102E20FEF78DF994F82B0018B9002115
:106ED0002D20FEF786F9FFF717FF04E0AFF6D80183
:106EE0002D20FEF7BFF9A06EF860E06494F836003C
:106EF00001286BD0FFF79AFBF968206F0144F96015
:106F0000E06494F83600022860D04DE074E064E05C
:106F1000657862616C6C00004404002020204853B6
:106F20005444000061776172642000003604002040
:106F30006164766E63650000470400206F707469B9
:106F40006F6E7300646F6E6500000000180700200C
:106F50006F7074696F6E0000A40200205804002056
:106F6000940400202504002090040020801A0600CC
:106F700070F305008404002098040020A40400207D
:106F8000B4020020D30B0020B80200202704002008
:106F90008C040020320400209C040020A80400205F
:106FA0008804002031040020FFF740FBF968A06F3F
:106FB0000144F960E06494F83600032806D0FFF736
:106FC00035FBF96838680144F960E064FFF72EFB8F
:106FD000FFF74EFEFCF7C9F85AE00C20D8F8001075
:106FE000FEF7FFF81620D8F80010FEF7FAF8D8F8E8
:106FF00000101C20FEF7F5F8F94800688047FEF7FE
:10700000AEFAF84800688047AFF60821F648FCF76A
:10701000ADFFF5490120FEF725F9F3490720FEF7FA
:1070200021F9F1491120FEF71DF9EF491720FEF76C
:1070300019F90620A16EFEF7D4F894F8360001285D
:1070400013D90C20216FFEF7CCF894F836000228F3
:107050000BD91620A16FFEF7C4F894F83600032868
:1070600003D91C203968FEF7BCF8FFF730F90FE0B0
:1070700048B9DE482671E570007802F0B1FC0421C1
:107080000020FEF7E7F9DA4800688047FEF723FFA3
:1070900094F84500022824D1D4481830007802F032
:1070A0009FFCD2482430007802F09AFC99F8000046
:1070B00002F096FC04F80D6F0C21E576257701208F
:1070C000FEF7C8F9FFF7C0FD01210020FEF756FECC
:1070D000C848007808B1FFF7C1FDBDE8F047FCF7EC
:1070E00044B8BDE8F08710B5FEF770F8FEF737FA40
:1070F00001210020FEF7AEF9BF48007830B1BF484B
:1071000001784FF030000029FEF76BF8B94800789D
:1071100008B1FFF7A3FDBA480078FFF73DFBB3497C
:10712000E83901F8320FB7480078FFF735FB4870AF
:10713000B5480078FFF730FB88700321BDE81040A8
:107140000120FEF787B970B50546FFF7D8FAA74CBE
:10715000E83C607E617D08430CD1AC480068804704
:10716000012084F8450094F83D006843BDE8704074
:1071700000F087B870BD70B5A5489C4D0078683D9B
:10718000A5F1800430B108210020FEF719FDE07E52
:10719000686470BD9F48007860B19F480068FFF741
:1071A000D2FF9E4800780028F1D005210220FEF78A
:1071B000E5FDECE7E17E686C8842E8D0984800780D
:1071C00010B1FFF7DCF901E0FFF725F894F8400073
:1071D000401C84F84000DAE7024692480168002922
:1071E0000FDD8A420BDD90480068884209DD82424B
:1071F00006DD8E490968814203DD8A4201DA0846CC
:1072000070470020704710B5784C894AE83C1168F7
:1072100094F83E00491C012811D002281AD00328F6
:1072200023D080346368002B2ADD2068984227DD54
:107230001160FFF7D1FF6060BDE810409BE7E36E8F
:10724000002B1DDDA06E98421ADD1160FFF7C4FF10
:10725000E066F1E7636F002B12DD206F98420FDDCF
:107260001160FFF7B9FF6067E6E7E36F002B07DD0A
:10727000A06F984204DD1160FFF7AEFFE067DBE727
:1072800086E570B5594DE83D2A4695F83E10927E48
:1072900005F18004012908D002290FD0032916D056
:1072A000216801442160DAB11DE0A96E0144A9669C
:1072B00012B90620FDF795FFA86E15E0296F01446D
:1072C000296712B90C20FDF78CFF286F0CE0A96F1D
:1072D0000144A96712B91620FDF783FFA86F03E0E8
:1072E0001C20FDF77EFF2068A0605248007868B13E
:1072F000A97D012009B1206108E04F4AA1689142AF
:1073000004DDA8753948183002F0A3FABDE87040D2
:1073100079E770B5354DE83DA87D00285FD0464E31
:10732000A96E05F18004B1420CDD2069B04204D1A0
:10733000AFF630510120FDF795FFA86E216990FB53
:10734000F1F1E9640620FDF74CFF296FB1420CDD35
:107350002069B04204D1AFF654510720FDF782FFF7
:10736000286F216990FBF1F1E9640C20FDF739FFEA
:10737000A96FB1420CDD2069B04204D1AFF67C5157
:107380001120FDF76FFFA86F216990FBF1F1E9640F
:107390001620FDF726FF2168B1420CDD2069B042BE
:1073A00004D1AFF6A0511720FDF75CFF21692068DA
:1073B00090FBF1F1E9641C20FDF713FF206901281F
:1073C00009D00A2190FBF1F0206108481830BDE88F
:1073D000704002F03EBA054826612430F7E72DE000
:1073E000A0020020AC020020D30B00208007002068
:1073F000A8020020370400203404002045040020A7
:10740000290400202A0400202B040020CC020020A4
:10741000220400202E040020A004002039040020B3
:107420002F0400208404002098040020A4040020DD
:10743000900400203504002040420F0070BDFF4939
:107440000020C87242F210707DE6FC4810B590F83A
:10745000430070B1012813D0022817D0AFF21051A9
:107460000120FDF7FFFEF6A1BDE810400720FDF763
:10747000F9BEF5A10120FDF7F5FEAFF67861F3E75F
:10748000F3A10120FDF7EEFEF3A1EDE7F4A1012049
:10749000FDF7E8FEF4A1E7E7E84890F82510012998
:1074A00001D0C16C01E0816DC1644165F049416664
:1074B000F049016642F21071C1657047704710B51E
:1074C000DE4C607E002843D194F8450002283FD06E
:1074D000E9480178E1B194F844000122401CC0B2AF
:1074E00084F8440081421CD1E4490868401C0860CB
:1074F000627602210120FDF7ADFF03210220FEF795
:107500003DFC042084F84500BDE81040FBF72DBE8B
:10751000022084F845000121BDE810400020FDF75D
:1075200099BFD748A276007802F05AFAD4480C30B6
:10753000007802F055FAD24802F08BF9D0480C30AE
:1075400002F087F9BDE81040CEA10120FDF78ABE08
:107550001EE4BA4991F84400002802D0401E81F888
:1075600044007047B54900208871704710B5B34C8E
:10757000207F0A280AD3142801D3E07F00E0A07FEF
:1075800084F82A00C1B20120FDF764FF207F0A21A0
:10759000B0FBF1F201FB1200A8498031002888619C
:1075A0000AD0617F0844401EC1B284F82A10BDE8A9
:1075B00010400120FDF74EBF62E610B59F4C207FC2
:1075C000142806D01D2804D00A2804D0132802D07D
:1075D00007E0E17F14E0A17F84F82A100020FDF786
:1075E00039FF207F0A21B0FBF1F201FB1200934921
:1075F0008031002888610AD0617F0844401EC1B2F2
:1076000084F82A10BDE810400020FDF723BF37E6BC
:1076100010B58A4C207F94F82D10884207D2FFF7CE
:10762000CCFF207F401C2077BDE810409EE727E676
:1076300070B5824C94F8200094F82C10884213D234
:1076400004F1CC05284410F8011C11B10020FDF70D
:1076500001FF94F82000295C11B10120FDF7FAFE2A
:1076600014F8200F401C207070BD70B5734D95F854
:107670002000012817D905F1CC04204410F8011C82
:1076800011B10020FDF7E6FE15F8200F401EC0B234
:107690002870204410F8011C002904D0BDE8704077
:1076A0000120FDF7D7BE70BD10B5644C042194F8DD
:1076B0002800F0B1312820D0401C84F8280094F82C
:1076C000290031281CD0401C84F8290014F8280F08
:1076D000FDF773FF20706078FDF76FFF6070217811
:1076E0000120FDF7B7FE6178BDE810400020FDF7EE
:1076F000B1BE84F828102D20E6E784F82810DEE7D4
:1077000084F82910E2E72DE9F0414C4C00250126D0
:1077100084F8255084F837600B205E4F84F83800D9
:107720005D490120FDF79EFD5B490720FDF79AFDAD
:1077300094F8370001280AD158A1FDF793FDAFF660
:107740008C410720FDF78EFD56480078E06494F8E0
:10775000370002280AD154A10120FDF783FD54A16E
:107760000720FDF77FFD54480068E06494F8370077
:1077700003280AD151A10120FDF774FD51A1072072
:10778000FDF770FD51480068E06494F83700042864
:107790000BD14AA10120FDF765FDAFF63851072056
:1077A000FDF760FD4A480068E06494F8370005285A
:1077B0000AD142A10120FDF755FD46A10720FDF7A2
:1077C00051FD46480068E06494F8370006280AD165
:1077D00032A10120FDF746FD41A10720FDF742FD42
:1077E00041480068E06494F8370007280AD13FA1B7
:1077F0000120FDF737FD3FA10720FDF733FD3F488E
:107800000068E06494F8370008280AD137A1012005
:10781000FDF728FD3AA10720FDF724FD3A4800684E
:10782000E06494F83700092878D130A10120FDF7F1
:1078300019FD36A10720FDF715FD6CE09806002024
:10784000736574757000000020646F6E6520000021
:107850002067616D6500000073746174730000003F
:10786000686172647772000074657374730000005D
:1078700080380100301B0F004604002074040020F3
:10788000B007002077686F616820627562626120CE
:1078900000000000940400200466000820746F7447
:1078A000616C000045040020202067616D650000C8
:1078B00073746172747300005804002020636F6950
:1078C0006E730000206C6566740000005C0400208C
:1078D000640400207269676874000000600400207E
:1078E0007265706C61730000700400206E756D62CB
:1078F00065720000736C616D730000006C04002001
:107900006562616C6C7300006804002074696C74BB
:107910007300000002E0F8480068E06494F8370063
:107920000A280ED1F5A10120FDF79CFCF5A1072046
:10793000FDF798FC3868E06494F82500022800D12F
:107940003D6094F8370094F83810884210D1EFA1C8
:107950000120FDF787FCAFF614210720FDF782FC1C
:107960004FF0FF30E565E06494F82500012818D059
:10797000E8491120FDF776FCE16C002902DB1620B6
:10798000FDF72FFCE448816C491E8164FEF70FFB74
:1079900084F8250001283FF4C3AE022807D003284D
:1079A0000AD0BDE8F041DB490720FDF75BBC606E03
:1079B000A06584F82560B3E694F8370094F8381091
:1079C000884202D184F83760AAE6401C84F8370068
:1079D000A6E6D148D149803890F83E00022801D867
:1079E000112000E00120FDF73DBC10B5CA4CC9498B
:1079F000803C94F83E00022816D81120FDF732FC96
:107A0000C4491720FDF72EFC94F83E00022803D944
:107A10001620A16FFDF7E5FB94F83E00032818D966
:107A2000BD4801681C2010E00120FDF71BFCB9498E
:107A30000720FDF717FC0620A16EFDF7D2FB94F896
:107A40003E00012805D9216F0C20BDE81040FDF74C
:107A5000C8BB15E410B5B2A10120FDF703FCB24884
:107A6000007808B1B1A100E0B2A10720FDF7FAFB50
:107A7000A94C803C94F82700E0B1B0A11120FDF79B
:107A8000F1FBA4491720FDF7EDFB94F8270098B10E
:107A9000012813D0AB4801681C20FDF7A2FB14F8A5
:107AA000270F401CC0B20321B0FBF1F201FB120012
:107AB00020704DE5A4A1E1E7A548ECE7A548EAE779
:107AC00070B5A54CA54E944D2068B04244DD2869A0
:107AD000B04213D18F499148FCF748FA8F490120F1
:107AE000FDF7C0FB8D490720FDF7BCFB8B4911203A
:107AF000FDF7B8FB89491720FDF7B4FB2068296919
:107B0000854C90FBF1F1803C0620E164FDF769FBB8
:107B10009348007868B393480168B14203DD28694F
:107B200091FBF0F1E1640C20FDF75BFB8E480168EE
:107B3000B14203DD286991FBF0F1E1641620FDF705
:107B400050FB8A480168B14203DD286991FBF0F1DE
:107B5000E1641C20FDF745FB2869012813D00A21A8
:107B600090FBF1F02861BDE870406B48743001F083
:107B700070BE0C20E16CFDF734FB1620E16CFDF7C4
:107B800030FBE16CE5E72E61EDE72DE9F047624C53
:107B9000803CA07B00287CD15E496048FCF7E6F978
:107BA00094F84500DFF8B49101255B4E4FF00008D2
:107BB000022811D0E17800296BD1042869D0A0797E
:107BC000A17D084365D1607B00287AD084F80D80C0
:107BD000A07E002876D01DE1A079002859D1644804
:107BE0000078002855D04D490120FDF73BFB4B495B
:107BF0000720FDF737FB49491120FDF733FB5D4FA7
:107C0000387818B945491720FDF72CFB42487430E5
:107C1000007801F0E5FE40488030007801F0E0FE99
:107C20003D488C30007801F0DBFE607BDFF848A136
:107C3000F8B184F80D800B210020FDF70BFC9AF8B9
:107C4000000030B1A07D20B1C6F81090FFF761FBB5
:107C5000A7E00620A16EFDF7C4FA0C20216FFDF706
:107C6000C0FA1620A16FFDF7BCFA387840BB316826
:107C700094E042486573007878B1A57094F82300C9
:107C8000401CC0B284F82300022808D9FFF7E2FEA6
:107C900000E0C6E084F8238083E084F802800B21B2
:107CA0000120FDF7D7FB9AF80000DFF8AC8050B157
:107CB000D8F80010494506DDC6F81090FFF700FF20
:107CC0006FE08AE070E00620D8F80010FDF789FA2E
:107CD0002348007870B1234801680C20FDF781FA31
:107CE000214801681620FDF77CFA387818B91F483A
:107CF000016853E044E054E074040020617665724A
:107D00006167000073636F7265200000202064616A
:107D1000746100000466000818070020D30B0020DF
:107D200020657874726100002F04002067616D6522
:107D30002020000062616C6C20200000616E6420D5
:107D400061740000A4040020202061742020000041
:107D500084040020980400208C04002040420F007E
:107D6000320400209C040020A80400208804002085
:107D7000330400203C0400203504002025040020AA
:107D80000C20D8F80010FDF72CFA1620D8F80010B7
:107D9000FDF727FA387820B9D8F800101C20FDF735
:107DA00020FAA571F74838E094F83E00012806D083
:107DB000022807D0032808D004282BD108E0F24974
:107DC000012007E0F049072004E0EF49112001E01D
:107DD000ED491720FDF746FA1CE06573C6F81090D0
:107DE000A07EB8B994F83E00012806D0022807D03A
:107DF000032808D004280DD108E00620A16E07E072
:107E00000C20216F04E01620A16F01E01C203168D6
:107E1000FDF7E7F9DB48A5710C30BDE8F04701F04C
:107E200018BDBDE8F0872DE9F05FD84D002401268C
:107E300085F82540D64FDFF85C93DFF85CA3DFF8C8
:107E40005C83DFF85CB385F82E60D6490720FDF728
:107E500009FA95F82E00012811D1AFF27051FDF703
:107E600001FAD1A10720FDF7FDF9D14B1878E8649C
:107E7000FEF782FC95F84C0018700820286695F8EB
:107E80002E0002280ED1CBA10120FDF7EBF9CBA1EA
:107E90000720FDF7E7F9CB4A1068E864FFF7FCFA22
:107EA000E86C106095F82E0003280ED1C6A10120C1
:107EB000FDF7D8F9C1A10720FDF7D4F9C44A10682D
:107EC000E864FFF7E9FAE86C106095F82E000428E2
:107ED0000ED1C0A10120FDF7C5F9B8A10720FDF71B
:107EE000C1F9BE4A1068E864FFF7D6FAE86C106082
:107EF00095F82E00052810D1B9A10120FDF7B2F99F
:107F0000AFF200210720FDF7ADF9D8F80000424696
:107F1000E864FFF7C1FAE86C106095F82E000628B7
:107F200012D1B1A10120FDF79DF9B1A10720FDF704
:107F300099F9B14B1878E864FEF71EFC95F84C00EF
:107F400018701E20C5E9180495F82E00072812D1D4
:107F5000AAA10120FDF786F9AAA10720FDF782F961
:107F6000AA4B1878E864FEF707FC95F84C001870E7
:107F70002820C5E9180495F82E00082811D1A44935
:107F80000120FDF76FF9A3A10720FDF76BF9DFF8DA
:107F90008CC29CF80000A870FEF7D6FBA8788CF87D
:107FA000000095F82E00092812D19949012048397E
:107FB000FDF758F99AA10720FDF754F9DFF868C2D8
:107FC0009CF80000A870FEF7BFFBA8788CF80000B2
:107FD00095F82E000A2823D18D490120FDF742F99A
:107FE00092A10720FDF73EF93878A870FEF7ACFBA8
:107FF0003878012812D1A87880B98E4AD8F80010B4
:1080000091420BDD8C49C8F800108C49C9F800106A
:108010008B49CAF800108B49CBF80010A87838704B
:1080200095F82E000B2813D1AFF290710120FDF7C7
:1080300019F985A10720FDF715F9854B1878E86433
:10804000FEF79AFB95F84C0018700520C5E9180456
:1080500095F82E000C2811D17EA10120FDF702F920
:108060007EA10720FDF7FEF8DFF8F8C19CF80000BC
:10807000A870FEF769FBA8788CF8000095F82E0030
:108080000D2811D178A10120FDF7ECF878A1072087
:10809000FDF7E8F8DFF8E0C19CF80000A870FEF7F3
:1080A00053FBA8788CF8000095F82E000E2811D10B
:1080B00072A10120FDF7D6F872A10720FDF7D2F8D2
:1080C000DFF8C8C19CF80000A870FEF73DFBA87857
:1080D0008CF8000095F82E000F2811D16CA101201A
:1080E000FDF7C0F86CA10720FDF7BCF8DFF8B0C1C0
:1080F0009CF80000A870FEF727FBA8788CF8000019
:1081000095F82E0095F83010884206D395F82F1078
:10811000884202D263480068804795F82E0095F89F
:108120002F1088420FD160A10120FDF79BF860A1BC
:108130000720FDF797F84FF0FF30EC65E86495F8FD
:10814000250001281AD017491120FDF78BF8E96C9A
:10815000002902DB1620FDF744F80C498031886CB9
:10816000401E886409D0FDF782FF95F8250001289C
:1081700005D0022804D0032803D09FE09CE0A8E0AB
:10818000DCE0E0E0C8070020D30B002098060020C8
:10819000350400209C040020A80400208C0400204A
:1081A000880400200466000862616C6C73000000A3
:1081B0002704002020666972737400007468726579
:1081C00073680000840400207365636F6E640000B0
:1081D000980400202074686972640000A4040020E0
:1081E000202068696768000020206175746F0000B6
:1081F00070657263656E00002504002020206261B6
:108200006C6C00007361766520200000260400205D
:10821000F46A00083420485354440000320400201B
:108220006873746420200000330400206D696C6959
:108230006F6E000040420F00E0E60B0020120A00C3
:10824000603D0800A068060074696C74732000002B
:10825000460400202069646C65200000616E696D31
:1082600061740000370400202066617374200000F0
:10827000626F6E75732000003004002020736B69FC
:108280006C6C000073686F74202000003B040020B9
:108290007475726E6D7400006D6F6465202000004F
:1082A00022040020C4020020207365747570000051
:1082B000646F6E652020000085F82E60AFF2180113
:1082C0000120FCF7CFFFBDE8F05FFD490720FCF778
:1082D000C9BFD5E91710421A686D824201DA686E8B
:1082E00000E00844A86595F82E00052823D1A86D64
:1082F00090FBF1F0484344F62061C8F80000884242
:1083000003DD411AC9F8001001E0C9F8004047F246
:108310003051884203DD411ACAF8001001E0CAF862
:10832000004049F64041884203DD401ACBF8000086
:1083300001E0CBF80040E348067086E5686EA8656A
:1083400085F82560F7E795F82E0095F82F108842FC
:1083500002D185F82E6078E5401C85F82E0074E582
:10836000D94910B50868D94C401C0860D84814F8A1
:10837000321F0078FEF797F92070D44C803401E06A
:10838000FDF726FF6069401E6061401CF8D110BDFA
:10839000D04910B50868CD4C401C0860CE4814F890
:1083A000341F0078FEF77FF92070C84C803401E05C
:1083B000FDF70EFF6069401E6061401CF8D110BDE2
:1083C000704770B500240D46224608E0295D04F18F
:1083D0000104E4B20029F9D102F10102D2B28242D1
:1083E000F4D304E0641CE4B20620FDF733F8295D01
:1083F0000029F7D170BDFDF7AABF10B5B34CE07BE3
:10840000002805D0FDF7ABF8FDF74EF90020E0732A
:1084100010BDB24810B50168AC4C491C0160B048B1
:10842000007818B114F8321FA94802E014F8331F7D
:10843000AC480078FEF737F92070A44C803401E096
:10844000FDF7C6FE6069401E6061401CF8D110BD9A
:108450009E4A012802F1800105D0022805D0032898
:1084600006D0086802E0906E00E0106F88607047E8
:10847000906FFBE72DE9F041044694481746884683
:1084800090F83E00FFF7E4FF904D80356426A86029
:1084900012E0A86890FBF6F106FB110068610A2063
:1084A000FEF751FE68695A280BD041460020FDF7BF
:1084B00065FCA8680A30A860641EE4B2E9D2BDE891
:1084C000F0813946F2E72DE9F04704467F489046AF
:1084D000894690F83E00FFF7BBFF7C4D4FF47A765B
:1084E00080354FF46177A86014E0A86890FBF6F13E
:1084F00006FB110068616420FEF725FE6869B8423A
:1085000001D1414600E049460020FDF737FCA8684C
:108510006430A860641EE4B2E7D282E42DE9F04141
:108520000F4604464FF47A766F4D09E03046FEF769
:108530000AFE39460020FDF721FC286801F013F8F7
:10854000641EE4B2F2D2BAE72DE9F0415F4C674D08
:10855000654FE0794FF47A7690B3207F84F841003C
:1085600094F8201004F1CC00084410F8011C0120FC
:10857000FCF770FF1FE094F841000FE0FEF7F6FFF4
:108580003046FEF7E0FD61780020FDF7F7FB286834
:1085900000F0E9FFFFF711F8207F401E207710F070
:1085A000FF0FEBD1386800F0DEFF94F820000128BF
:1085B00007D9FFF75AF894F820000028DBD17EE7AE
:1085C00022E0002084F8200079E7FEF7CFFF94F83E
:1085D00020000CE03046FEF7B6FD61780020FDF784
:1085E000CDFB286800F0BFFF94F84100401E84F8DE
:1085F000410010F0FF0FEDD1FEF7DFFF207F401E9E
:108600002077386800F0AFFF207F0028DDD156E7E3
:108610007047374810B50168491C01602B4902209A
:1086200081F8450001210020FCF714FF0221012000
:10863000FCF710FFFCF7CAFDFDF74DFC2DA1012052
:10864000FCF710FE2DA10720FCF70CFE00F0A9FF9F
:1086500001F04BF82B490020086003210220FDF7B0
:108660008DFBFAF782FD41F2883000F05BFF26486F
:108670000068BDE81040004710B58AB006281AD23D
:10868000DFE800F019030D76818C20A10120FCF7B2
:10869000E9FD20A10720FCF7E5FD20A108E024A1C9
:1086A0000120FCF7DFFD24A10720FCF7DBFD24A15E
:1086B0006846FBF75BFC2748007803284FD34BE064
:1086C00004660008A60800205C040020980600202C
:1086D00029040020640400202B04002060040020F2
:1086E000280400202A040020500400204C0400200C
:1086F0006C0400202020626164200000206F6E6501
:108700002020000034090020A4020020737769743F
:10871000636800006F7672666C6F0000537769744F
:1087200063682051204F766572666C6F7700000099
:108730007174696D65720000777463686467000026
:1087400054696D6572205461626C652066756C6C4D
:1087500000000000D00300206846FBF78CFBED4CC6
:108760008020012184F845000020FCF773FE22E000
:10877000E9A10120FCF776FDAFF244010720FCF7E8
:1087800071FDE7A194E7EBA10120FCF76BFDAFF2CF
:1087900058010720FCF766FDE8A189E7ECA101205C
:1087A000FCF760FDAFF270010720FCF75BFDEAA16A
:1087B0007EE7FDF790FBFDF7A9FB7028F9D10220B9
:1087C00084F845000AB010BD10B5D24C4FF00B0133
:1087D000A07808B1012000E00020FCF73BFEA07863
:1087E00010B10020A07010BD0120FBE7C948417CFA
:1087F00011B100214174704701214174DC480068C7
:10880000004710B5142839D2DFE800F0380A0D11FE
:1088100013161A1D2020232629292D3033353B3BE2
:10882000FDF754FE2DE0D3480068804729E0D24888
:1088300003E0FFF7E2FD24E0D0480068804720E035
:10884000FDF75AFE1DE0FFF73BF91AE0FEF761FD68
:1088500017E0FEF77EFE14E0FEF77DFA11E0AD4969
:10886000002088710DE0FFF7C1FF0AE0FDF76FFD02
:1088700007E0C348E1E7FFF7A7FF02E0C149096845
:108880008847002010BD10B5703808281ED2DFE8D8
:1088900000F004070A0D1013161900F04BFD13E049
:1088A000FFF75EFD10E0FFF7B4FD0DE0FFF770FD90
:1088B0000AE0FDF74CFD07E0FEF701FE04E0FEF7DD
:1088C00068FA01E0FFF7A5FE002010BD4FF0FF3071
:1088D00010BD70B5AC480024AE490470AB4801250A
:1088E0000470AB48047005200870AB48B1A1057056
:1088F000AA480460AA480460AA480460AA4805700F
:10890000AA480570AA480570B148FBF72FFBB1488B
:10891000B449CE4A0470B048D24B0470AF480570D9
:10892000AF48057040F6C4100860AF48B149047004
:10893000AE480470AE480860B049AF480860B0481F
:10894000B1490460AF480860B048B3490570B04809
:108950000570B04805700F200870B048B049047029
:1089600003200870AF490C70AF490C60AF490C6030
:10897000AF490C60AF490C60AF490C60AF490D7056
:10898000AF490C60AF490D70AF491160B14AB049B1
:108990001160B14A1470B14A1470B14A157044F6AE
:1089A00020621A60B04A1470B04B4FF47A721A60A9
:1089B000AF4BC8221A70AF4A1160B04AAE4911607D
:1089C000AF490870AF4946200860AF495F20086092
:1089D000AE48B1490470AE480470AE4804706420DB
:1089E0000860AE49DC20086070BDF0B5AC480123DA
:1089F000AC4906780020AC4AAC4CAD4D0C2E11D2DF
:108A0000DFE806F010061113061511091310191DE1
:108A10000870107005E0A74912200870A649087078
:108A200032202070F0BD2870F0BD0B7005E008709A
:108A300028702370F0BD287008701370F0BD0870A6
:108A4000F0BD2DE9F041334C324F0126803704F858
:108A5000026F00257D61BD61C4F84A50C4F84E50D4
:108A600096A198481E34FBF781FA04F81D5C04F8BF
:108A70001A5C4FF00F0804F8038C66700A20A0708F
:108A800004F8195C6563E5702571A563657104F8E8
:108A9000165C022084F8250004F8145C04F8136CBA
:108AA00004F8125C85A107F15100E563FBF75EFA5B
:108AB0007D6225726572A57204F8115C84F80D80E0
:108AC0002564A6731020207465646574A674E6742A
:108AD000267584F81580E67584F818804FF4487080
:108AE000B86240103862FA20F862E57776A1A7F103
:108AF0003A00FBF73BFAFD6004F8105C04F80E5CEA
:108B000004F80B5C84F822504FF41670B86404F833
:108B1000155CD4E498060020716576656E740000DB
:108B20004576656E74205461626C652066756C6C68
:108B300000000000636576656E740000436F756C1D
:108B4000646E7420636C656172206576656E740076
:108B5000756576656E740000436F756C646E742085
:108B60007570646174652074696D65720000000041
:108B7000D0020020A4020020C8020020BC02002075
:108B8000D4020020880200202404002025040020B4
:108B90002604002027040020280400205C04002074
:108BA0006004002064040020290400202A0400201E
:108BB0002B04002053797374656D38302043505571
:108BC000202041524D20206D6F64656C0000000034
:108BD000430B00202C04002032040020330400202A
:108BE00034040020540400203504002047040020F1
:108BF000C0D4010084040020708203008804002097
:108C00005804002000E204008C04002036040020F8
:108C100037040020310400204204002043040020D7
:108C20004404002045040020680400206C04002057
:108C300070040020900400207404002039040020F7
:108C4000940400203A04002020BF02009804002071
:108C5000C04504009C0400203B0400202E0400209A
:108C60002F040020A00400203004002078040020FD
:108C70002D040020A404002090D00300A8040020AC
:108C8000460400204C040020500400203C04002036
:108C9000220400203D0400207C04002080040020E9
:108CA0004804002020040020210400203F0400206C
:108CB0003E04002040040020410400206E756C6CCE
:108CC00000000000D30B0020312E323700000000DE
:108CD00010B5FDF72DF9FF280AD0FDF729F9702806
:108CE00008D0742806D0FDF711F9FF49002008705C
:108CF000002010BD012010BD2DE9F041FB4FFC4DBF
:108D00004FF49678C7F800802878012405F13306DF
:108D1000002871D0C0EBC00081190720C91FFCF7E3
:108D2000A1FA27E0FDF743F9012804D0022852D028
:108D300003281FD153E0EC49002008702878072849
:108D400018D2DFE800F048040C0F1215220024B1FD
:108D500000242046FCF7C7FA0CE00124F9E7FCF7F1
:108D6000B3FC07E0FCF777FF04E0FDF799F901E0B9
:108D7000FDF72AF83868401E3860401CD2D1DD4922
:108D8000022008700120BDE8F081FFF7A2FDDA485B
:108D9000DA4A0068A0F59C4120391160D84AA0F554
:108DA000EA4130391160D749A0F51C4040380860CD
:108DB0000120687003210020FCF702FFCC49072046
:108DC000891CFCF74FFA4FF4FA7000F0CCFBC8494D
:108DD0004F310720A3E7FCF7F9F90020D3E7C7F8E4
:108DE0000080287801240721401CB0FBF1F201FB30
:108DF000120028708CE7FFE7BD49891C07208EE729
:108E00002DE9F041B94C4FF49670BF4D2060BFA1E1
:108E10002F780720FCF726FADFF8F882297811204E
:108E200058F82110FCF71EFA002640E0FDF7BFF8C5
:108E3000012804D0022812D0032838D112E0B64805
:108E40000C2106702878401CB0FBF1F201FB1200E7
:108E5000287058F820101120FCF704FA27E02E7033
:108E6000002090E7ADA10720FCF7FCF9ABA117208B
:108E7000FCF7F8F92878B84218D09D4901204870CD
:108E8000FAF7E7F890B9A748008881B2A6480078B9
:108E900000F0F6FDA548008881B2A548007800F0F2
:108EA000EFFDFFF7A2FDA348006880472660206819
:108EB000401E2060401CB9D1012064E72DE9F05F1D
:108EC00001249D4900209D4DDFF874829D4E9E4FE8
:108ED0004FF00C0AA146087090A10720FCF7C2F9D8
:108EE000012C49D0022C52D0032C69D0042C7DD007
:108EF000052C7CD0062C7BD0072C7AD0082C79D07E
:108F0000092C78D00A2C77D00B2C76D0544510D170
:108F10008EA10120FCF7A6F98EA10720FCF7A2F98B
:108F20004FF0FF302860002030608348007801282F
:108F300018D07AA11120FCF795F92968002902DBE5
:108F40001620FCF74EF969490868401E086009D0F0
:108F5000FDF78DF87849087801287DD002287CD06B
:108F600003287BD079A10120FCF77CF9BDE8F05FF4
:108F70006AA10720FCF776B978A10120FCF772F905
:108F800078A10720FCF76EF9DFF8E0B109E078A1DD
:108F90000120FCF767F973A10720FCF763F9DFF8FC
:108FA000D8B1DBF800002860FDF7E6FB29681E2039
:108FB000CBF800103860A020C8F8000005203AE186
:108FC0006EA10120FCF74EF96EA10720FCF74AF9CB
:108FD000DFF8B8B19BF800002860FDF7CDFB2878DA
:108FE0008BF8000064204FF4967107E00AE022E05D
:108FF00040E061E0F2E005E11FE133E13860C8F8EC
:109000000010DBE762A10120FCF72CF962A1072028
:10901000FCF728F9DFF888B19BF800002860FDF71D
:10902000ABFB28788BF800000A2032213860012041
:10903000C8F80010FFE05BA10120FCF713F95BA169
:109040000720FCF70FF9DFF86CB1DBF800002860AF
:10905000FDF792FB296802E04EE15CE163E1CBF8A9
:1090600000104FF42F70386040F2DC516420C8F8D3
:109070000010E0E050A10120FCF7F4F84BA107201C
:10908000FCF7F0F8DFF8A4B0DBF800002860FDF78B
:1090900073FB2868CBF8000081B22548007800F007
:1090A000EFFC21499BF800000870C820410038609F
:1090B0001420C8F80010BEE041A10120FCF7D2F84E
:1090C0003AA10720FCF7CEF8DFF858B0DBF8000033
:1090D0002860FDF751FB2868CBF8000081B21248E8
:1090E000007800F0CDFC6FE02C0900203009002052
:1090F000A5080020DD0600208C0400209C04002030
:10910000A8040020880400204804002073656C65D2
:109110006374000038080020240400202020202050
:10912000202000007C040020740700208004002020
:10913000EC0700208C020020BD060020E406002081
:10914000F8060020F4060020FC0600206578706513
:1091500072740000646F6E65202000002073636FDE
:10916000726500006C616720746D0000500400207F
:1091700020626F6E757300004C0400202020636F26
:10918000696C0000686C6420746D00002D04002080
:1091900020206C616D700000656E6120746D0000B0
:1091A000420400207377697463680000737472204E
:1091B000746D000078040020666C617368670000BD
:1091C000706620616E690000AD489BF80010017068
:1091D00050203860C820C8F800002BE0A9A1012069
:1091E000FCF740F8A9A10720FCF73CF8A948DFF8F4
:1091F000A8B201788BF80010FDF7A6FA9BF80010D2
:10920000A4482DE0AFF264010120FCF72BF8A3A1E4
:109210000720FCF727F8DFF88CB29BF800002860E5
:10922000FDF7AAFA28788BF800001E2096213860F6
:10923000C8F800100A2030607BE69BA10120FCF7F3
:1092400011F89BA10720FCF70DF89B48DFF848B206
:1092500001788BF80010FDF777FA9BF8001096481C
:10926000017066E695A10120FBF7FCFF95A10720A0
:10927000FBF7F8FFDFF820B25FEA09008BF80090F7
:109280001BD092A11120FBF7EDFFDFF848920DE013
:109290000B210120FCF7DEF8642000F064F90B21BB
:1092A0000020FCF7D7F8642000F05DF98A48D9F86F
:1092B000001000688142EBD019E088A11120FBF773
:1092C000D1FF884800F0C5FADFF8089205E086482B
:1092D0000078022801D100F000FB7F48D9F8001087
:1092E00000688142F3D07F48007800F079FBFDF7F9
:1092F0002BFA9BF800901CE6D8F8001030680A1A88
:109300007A4909688A4201DA386800E008447849F5
:109310000860012004E0764A386810600120087077
:1093200074494870D8E5544501D10124D4E5641C42
:10933000E4B2D1E52DE9F05FDFF8BCB120210020D7
:109340008BF800100121FCF785F8FBF73FFFFCF7D5
:10935000C2FD00F0CAF969494FF00009DFF894A195
:10936000C1F8009001218AF800100D464FF41678DC
:109370000AF102068AF801904446F11D44E0FCF728
:1093800016FE012804D002282DD003283FD12CE05E
:10939000C5EBC50081190F460120FBF763FF072DC0
:1093A00016D2DFE805F02004070A0D101300FEF7BF
:1093B0003AFD0DE0FEF7A7F90AE0FFF79DFC07E094
:1093C000FDF7F6F904E0FFF71BFD01E0FFF776FD7E
:1093D000002C08DD444639460120FBF743FFAFF27D
:1093E000C421112011E0002411E045486D1C4446C1
:1093F0000078EDB208B1072000E00620A84200D1B5
:109400000025C5EBC50081190120FBF72BFF201EAD
:10941000A4F10104B3DC9AF80100544658B139A113
:109420000120FBF71FFF39A10720FBF71BFFF9F70E
:109430009CFE84F801904FF4487000F094F80225E7
:109440005C468BF80050FBF7C1FE3248007828B12B
:10945000314801783020FBF7C4FE04E0AFF2403120
:109460002F20FBF7FFFE2D4801782E20FBF7B9FED9
:109470002B49257081F80090BDE8F05FFDF733BE01
:1094800074070020656E61626C650000546465625B
:10949000756700003C0400209A0600206475702067
:1094A000746D00003408002064697361626C000010
:1094B00020536C616D2000003D0400202020546981
:1094C0006D65000063616C696272000020776169FC
:1094D00074200000700600207406002020636F7264
:1094E0006520000028080020CF030020EC060020A3
:1094F000F0060020A5080020DD0600203409002029
:1095000047040020736176696E6700006E767261B1
:109510006D200000340400204504002031040020A8
:109520009E06002001B582B00020FE49087001208F
:10953000019012E00120009007E0FA48007808B19D
:1095400001980EBD0098401C009040F678210098CC
:109550008842F2D90198401C0190DDE9010188425E
:10956000E8D90020EDE701B583B00120029013E0B7
:109570000120019008E0EB48007810B140F624602B
:1095800000900198401C019040F678210198884293
:10959000F1D90298401C0290DDE902018842E7D926
:1095A0000FBD0020E0490880E0490870E0490870DC
:1095B000E049087040F26D10DF4908800420DF495F
:1095C00008707047DD480078DD4908700520DB49E8
:1095D00008707047DA480078D849087070474188A9
:1095E000D14A11808179D14A11704179D04A1170E4
:1095F0000179D04A11700188CF4A1180D14AC168DF
:1096000011600321CD4A11707047CF480088CF49BF
:109610000880CF4800780871CE4800784871CE485D
:1096200000788871CD4800884880704700B50346AF
:10963000FFF7EBFFC54840881844801E82B24FF404
:109640007A7092FBF0F100FB1120C04948804FF482
:109650007A7092FBF0F082B2002A34DD08468079FD
:10966000104482B23C2092FBF0F100FB1120B7497C
:1096700088713C2092FBF0F082B2002A23DD08467C
:109680004079104482B23C2092FBF0F100FB1120A3
:10969000AE4948713C2092FBF0F082B2002A12DD04
:1096A00008460079104482B2182092FBF0F100FBCA
:1096B0001120A6490871182092FBF0F082B20846EA
:1096C00000881044088000BD9B4800889F4908809E
:1096D0009848007808719648007848719348007857
:1096E00088719148008848807047002008E0002178
:1096F00000EB40029A4B03EBC2021172411CC8B24C
:109700002028F4DB0021974A11607047014611B907
:109710004FF0FF30704708888B4B1B88181A924B0C
:1097200000FB03F208798A4B1B78181A4FF4616327
:1097300003FB00224879874B1B78181A3C2303FB54
:1097400000228879844B1B78181A02444888834B7E
:109750001B88984200DD521E802A02DD4FF0FF3048
:10976000D8E710B2D6E7024602B111B96FF0020095
:10977000704710880B88984201DD0120F8E71088B7
:109780000B88984202DA4FF0FF30F1E710790B793D
:10979000984201DD0120EBE710790B79984202DA5B
:1097A0004FF0FF30E4E750794B79984201DD01201A
:1097B000DEE750794B79984202DA4FF0FF30D7E775
:1097C00090798B79984201DD0120D1E790798B79EE
:1097D000984202DA4FF0FF30CAE750884B8898422F
:1097E00001DD0120C4E750884B88984202DA4FF02F
:1097F000FF30BDE70020BBE72DE9F041044600271C
:109800005848056801E02E466D6929462046FFF755
:10981000AAFF002804DD3846791CCFB2FA28F2DB13
:10982000FA2F02DB0220FEF727FF4E480068854230
:1098300002D04C48006840B94A4800686061494815
:1098400004600068FFF7CBFE01E074616561BDE86C
:10985000F0812DE9F04104460027A0880A2802DAA9
:10986000781EBDE8F081002601E0701CC6B2202EF3
:109870000BDA06EB46003A4901EBC000007A20B152
:109880003846791CCFB2FA28EFDBFA2F02DB03202F
:10989000FEF7F2FE202E02D14FF0FF30E1E706EB9B
:1098A00046002F4901EBC005A088FFF7BFFE2748FF
:1098B000016829608188A9808079A871A0882882A0
:1098C00060786872A078E87120782872A068E860F3
:1098D0002846FFF791FF0020C3E710B54FF0FF3097
:1098E0002249096808601F480068002860D01D48A8
:1098F00000681F4908600846006840691949086007
:1099000006200E4908701A490968487AFEF779FF5F
:1099100017480068C07901282CD100201449096833
:10992000087245E02C090020180900201A090020BF
:109930001B0900201C0900201E090020CF03002065
:109940003C090020440900200E090020640F00207B
:109950000C0900200B0900200A090020080900203A
:10996000640C0020340900208051010024090020EB
:109970004009002054480068C079002806DD52489C
:109980000068C079401E50490968C8714E4909688D
:10999000088AFFF74BFE4C4800684C490A68026091
:1099A0008A8882808979817147480068FFF724FF9F
:1099B0004748006818B90420464908700CE044483C
:1099C000006841490968884203D041480068FFF7B0
:1099D00006FE03203F49087000203B49086010BD87
:1099E0002DE9F04705464FF00009C84636480068A3
:1099F00040B135480068007AA84203D101203249BD
:109A00000968C8713248006810B94846BDE8F08757
:109A10002F480468274616E0207AA84201D026463F
:109A200010E04FF001092A480068A04206D1062044
:109A30002849087026496069086001E06069706122
:109A40000020207264692CB14046411C01F0FF08DF
:109A50006428E1DBB8F1640F02DB0420FEF70CFEA2
:109A60001B480068B84204D019480068FFF7B7FDEA
:109A700004E01748006808B9FFF793FD4846C5E7BA
:109A80002DE9F04105460E464FF00008002710482A
:109A9000006810B94046BDE8F0810D48046806E052
:109AA000207AA84202D14FF001082682646924B1CD
:109AB0003846791CCFB2FA28F2DBFA2F02DB0520F8
:109AC000FEF7DAFD4046E6E740090020640F00207B
:089AD00034090020CF0300203F
